:020000040000FA
:100000006028900B0128080005309300063092000C
:10001000920B0828930B062808000420910B0D284A
:1000200008002F0889002E088800831608158B13F6
:1000300055308900AA308900881488181D280811B5
:10004000831208002F0889008316081483120808F9
:10005000AE000800051A35280518970A8518970B71
:100060000519960A8519960B4B280518950A8518C7
:10007000950B4B281508AE000130AF001120160873
:10008000AE000230AF0011201708AE000330AF0001
:1000900011204B20080004308C000000FF3091003C
:1000A0000D208C0B4D280800143095000A30960066
:1000B000AE0005309700AE00283098002A2088282E
:1000C0008316103086001F3085008312FF308600B3
:1000D000051A54280130AF0022202E089500023066
:1000E000AF0022202E0896000330AF0022202E08F9
:1000F00097002830980088281508900006100120E5
:1001000006140800170890008611012086150800C3
:100110007C201608900001208220180891000D20F4
:1001200005182A2085182A2005192A2085192A2031
:10013000061A3A208828FF3FFF3FFF3FFF3FFF3F5F
:10014000FF3FFF3FFF3FFF3FFF3FFF3FFF3FFF3FBF
:10015000FF3FFF3FFF3FFF3FFF3FFF3FFF3FFF3FAF
:10016000FF3FFF3FFF3FFF3FFF3FFF3FFF3FFF3F9F
:10017000FF3FFF3FFF3FFF3FFF3FFF3FFF3FFF3F8F
:084000008F3FFF3FFF3FFF3F30
:02400E00F23F7F
:10420000FF003E0005000400FF00FF00FF00FF006C
:10421000FF00FF00FF00FF00FF00FF00FF00FF00A6
:10422000FF00FF00FF00FF00FF00FF00FF00FF0096
:10423000FF00FF00FF00FF00FF00FF00FF00FF0086
:10424000FF00FF00FF00FF00FF00FF00FF00FF0076
:10425000FF00FF00FF00FF00FF00FF00FF00FF0066
:10426000FF00FF00FF00FF00FF00FF00FF00FF0056
:10427000FF00FF00FF00FF00FF00FF00FF00FF0046
:00000001FF
